:020000040000FA
:100000008301372800000000F000030E8301F10097
:100010000408F2000B1D30280B1183120313AB0FE1
:10002000142883120313AC0A83120313B10F1B2885
:1000300083120313B20A83120313B40F222883120C
:100040000313B50A83120313B60F2928831203136F
:10005000B70A83120313B80F302883120313B90AA7
:1000600072088400710E8300F00E700E09002030BB
:100070008B008312031300308500003086000F30A0
:10008000831603138100FB308500FF308600831246
:10009000031307309F008313203084008001840AFB
:1000A000841F4E2884168001840AF0300402031D48
:1000B00053288317203084008001840A50300402C2
:1000C000031D5C28803083120313A20083120313E4
:1000D00081010B118B1783120313271D73288312C1
:1000E0000313A001892883120313A21D89288312F8
:1000F0000313211889288312031321148312031375
:100100002218862883120313A00A89288312031356
:10011000A00383120313A219902883120313211042
:1001200083120313A21C9C2883120313221D9F28F1
:100130008312031322149F288312031322108312A5
:100140000313A21CAC28831203132318AC28231416
:1001500083120313A215B62883120313A21183126C
:100160000313A218B6288312031323108312031358
:10017000271DBE2883120313A401D428831203135E
:10018000221ED428831203132518D42883120313A4
:100190002514831203132218D12883120313A40AEF
:1001A000D42883120313A40383120313221ADB2817
:1001B00083120313251083120313A219E728831255
:1001C0000313A21AE728831203132212EA288312C8
:1001D00003132216831203132219F7288312031321
:1001E0002618F728261483120313A2160129831256
:1001F0000313A21283120313221D01298312031376
:10020000261083120313221B0E29831203132818AE
:100210000E29281483120313A71518298312031318
:10022000A71183120313221F182983120313281006
:1002300083120313A21F25298312031329182529CA
:1002400029148312031322172F2983120313221355
:1002500083120313A21B2F29831203132910831265
:100260000313A21700308312031324028312031313
:10027000031D3C2927143D29271001308312031345
:10028000200283120313031D4729A7144829A7102E
:1002900083120313271C542983120313A71C542908
:1002A000831203132716572983120313271283126D
:1002B0000313271A6F2983120313A71A6F298312B6
:1002C0000313A7196F2983120313AA186F29831226
:1002D00003132A196F29831203132711722983121A
:1002E0000313271500308312031320028312031314
:1002F000031C7E2903197E29A7177F29A713FE3027
:1003000083120313200283120313031C8929A716E7
:100310008A29A712003083120313240283120313C5
:10032000031C962903199629271797292713831247
:100330000313A71BA72983120313271BA7298312C3
:1003400003133018A729831203132A10AA29831232
:1003500003132A14FE30831203132402831203139F
:10036000031CB429AA14B529AA1083120313AD18CB
:10037000CD29831203132D18DF2983120313AA1D1D
:10038000DF2983120313AB0183120313AC01831221
:100390000313AD14831203132A15073083120313BA
:1003A0002C02031DD729A130831203132B02031C37
:1003B000DF2983120313AD10831203132A11831252
:1003C0000313AA1DE729831203132D14EA298312AC
:1003D00003132D1083120313AA1EF2298312031391
:1003E000AE01FD29831203132F18132A831203135E
:1003F0002A1D132A83120313AE0A831203132E1C21
:10040000052A831203133014082A831203133010B1
:1004100083120313AE1C102A831203132A16132A05
:10042000831203132A12831203132A1D1B2A831219
:1004300003132F141E2A831203132F108312031386
:100440002A1B2A2A831203132A1A2A2A8312031325
:10045000AA122D2A83120313AA1600308312031343
:10046000200283120313031D372AAA17382AAA135E
:1004700083120313B318502A831203133318622A0A
:1004800083120313AA1F622A83120313B10183127A
:100490000313B20183120313B314831203132A1735
:1004A0000030831203133202031D5A2A4E30831286
:1004B00003133102031C622A83120313B310831245
:1004C00003132A1383120313AA1F6A2A8312031326
:1004D00033146D2A831203133310831203132A1863
:1004E0007B2A83120313B40183120313B501831211
:1004F0000313B0108E2A83120313B0188E2A003013
:10050000831203133502031C8E2AC3308312031394
:100510003402031C8E2A83120313B01483120313B4
:10052000851C962A83120313B015992A831203138C
:10053000B01183120313051CA12A83120313301573
:10054000A42A83120313301183120313851DAC2ACE
:1005500083120313AA15AF2A83120313AA1183125D
:100560000313B01CB72A831203130515BA2A83128A
:1005700003130511831203133019C82A83120313BE
:10058000B60183120313B701831203132211DB2A6E
:10059000831203132219DB2A01308312031337025B
:1005A000031CDB2A3830831203133602031CDB2AB8
:1005B00083120313221583120313B019E92A83123D
:1005C0000313B80183120313B90183120313A2109A
:1005D000FC2A83120313A218FC2A0130831203138E
:1005E0003902031CFC2A3830831203133802031C1F
:0A05F000FC2A83120313A2146B28E7
:084000000000010000000000B7
:02400E00613F10
:00000001FF
